:020000040800F2
:1000000014040020250100088D0100088D0100085E
:100010008D0100088D0100088D010008000000001E
:100020000000000000000000000000008D0100083A
:100030008D010008000000008D0100088D010008FE
:100040008D0100088D0100088D0100088D01000858
:100050008D0100088D0100088D0100088D01000848
:100060008D0100088D0100088D0100088D01000838
:100070008D0100088D0100088D0100088D01000828
:100080008D0100088D0100088D01000800000000AE
:100090000000000000000000000000008D010008CA
:1000A0008D0100088D0100088D0100088D010008F8
:1000B0008D0100088D0100088D0100088D010008E8
:1000C0008D0100088D0100088D0100088D010008D8
:1000D0008D0100088D0100088D0100088D010008C8
:1000E0008D0100088D0100088D010008000000004E
:1000F0000000000000000000000000000000000000
:1001000000000000000000000000000000000000EF
:1001100000000000000000008D0100088D010008B3
:100120005FF808F180B582B000AF134B7B60134BD2
:100130003B600BE07B681A683B681A603B6803F120
:1001400004033B607B6803F104037B603A680C4B5B
:100150009A42EFD30B480C494FF000028842B8BFD7
:1001600040F8042BFADB00F015F800F05FFA07F115
:100170000807BD4680BD00BF1C0C00080000002021
:1001800014000020140000201400002080B400AFF0
:10019000FEE700BF80B500AF174B174A126842F068
:1001A00001021A60144A144B5968144B01EA030304
:1001B0005360114A104B1B6823F0847323F480337F
:1001C00013600D4B0C4A126822F480221A600A4B0D
:1001D000094A526822F4FE025A60074B4FF41F028C
:1001E0009A60054B4FF00002DA6200F00BF8044B06
:1001F0004FF000629A6080BD001002400000FFF8DE
:1002000000ED00E080B500AF00F002F880BD00BF57
:1002100080B483B000AF4FF000037B604FF0000369
:100220003B60314B304A126842F480321A602E4BE8
:100230001B6803F400333B607B6803F101037B60C0
:100240003B68002B03D17B68B3F5A06FEFD1264B41
:100250001B6803F40033002B03D04FF001033B6015
:1002600002E04FF000033B603B68012B37D11E4B8F
:100270001D4A52685A601C4B1B4A52685A601A4BFE
:10028000194A52685A60184B174A526822F47C1275
:100290005A60154B144A526842F498125A60124B35
:1002A000114A126842F080721A6000BF0E4B1B6840
:1002B00003F00073002BF9D00B4B0B4A526822F06D
:1002C00003025A60084B084A526842F002025A6020
:1002D00000BF054B5B6803F00C03082BF9D107F155
:1002E0000C07BD4680BC70470010024080B489B046
:1002F00000AF786039604FF00003FB614FF00003FE
:100300003B614FF00003BB614FF00003FB604FF017
:1003100000037B614FF00003BB603B68DB7803F0B8
:100320000F03FB613B68DB7803F01003002B05D063
:100330003B689B78FA6942EA0303FB613B681B88D0
:1003400003F0FF03002B51D07B681B687B614FF0EB
:100350000003BB6144E0BB694FF0010202FA03F302
:10036000FB603B681B881A46FB6802EA03033B619B
:100370003A69FB689A422FD1BB694FEA8303FB605D
:10038000FB684FF00F0202FA03F3BB60BB686FEA31
:1003900003037A6902EA03037B61FB68FA6902FAE4
:1003A00003F37A6942EA03037B613B68DB78282B1D
:1003B00007D1BB694FF0010202FA03F27B685A6170
:1003C0000AE03B68DB78482B06D1BB694FF001029D
:1003D00002FA03F27B681A61BB6903F10103BB6196
:1003E000BB69072BB7D97B687A691A603B681B88A1
:1003F000FF2B56D97B685B687B614FF00003BB61C4
:1004000049E0BB6903F108034FF0010202FA03F36C
:10041000FB603B681B881A46FB6802EA03033B61EA
:100420003A69FB689A4232D1BB694FEA8303FB60A9
:10043000FB684FF00F0202FA03F3BB60BB686FEA80
:1004400003037A6902EA03037B61FB68FA6902FA33
:1004500003F37A6942EA03037B613B68DB78282B6C
:1004600008D1BB6903F108034FF0010202FA03F25D
:100470007B685A613B68DB78482B08D1BB6903F184
:1004800008034FF0010202FA03F27B681A61BB69AC
:1004900003F10103BB61BB69072BB2D97B687A69A1
:1004A0005A6007F12407BD4680BC704780B487B00E
:1004B00000AF78600B46FB704FF000033B614FF0DC
:1004C0000003FB604FF000037B614FF00003BB6053
:1004D0007B68002B03DA354BDB697B6102E0334B31
:1004E0005B687B617B6803F470234FEA1343BB6056
:1004F0007B684FEA03434FEA13433B617B6803F495
:100500004013B3F5401F0AD17B6923F070637B6110
:10051000264B264A526822F070625A6028E07B68B7
:1005200003F48013002B11D0BB684FF0030202FAD2
:1005300003F3FB60FB686FEA03037A6902EA0303D3
:100540007B617B6943F070637B6111E07B684FEAFC
:1005500053534FEA03133A6902FA03F36FEA0303B2
:100560007A6902EA03037B617B6943F070637B6114
:10057000FB78002B0BD07B684FEA53534FEA0313F1
:100580003A6902FA03F37A6942EA03037B617B6802
:10059000002B03DA054B7A69DA6102E0034B7A69D2
:1005A0005A6007F11C07BD4680BC7047000001403F
:1005B00080B483B000AF0346FB7100BF074B1B88BC
:1005C0009BB203F04003002BF8D0044BFA7992B2AF
:1005D0009A8007F10C07BD4680BC70470038014087
:1005E00080B584B000AF78604FF00003FB730AE081
:1005F000FB7B7A68D3181B781846FFF7D9FFFB7B83
:1006000003F10103FB73FB7B7A68D3181B78002B83
:10061000EED14FF00D00FFF7CBFF4FF00A00FFF7D0
:10062000C7FF07F11007BD4680BD00BF80B586B08B
:1006300000AF44F20D004FF0010100F0BDF9774822
:100640004FF00101FFF732FF40F2FF333B824FF0E2
:100650001003FB744FF00203BB7407F110037048E2
:100660001946FFF743FE6E4B4FF00002DA604FF47D
:1006700080633B824FF00403FB7407F11003694869
:100680001946FFF733FE4FF400733B824FF003032C
:10069000BB744FF01803FB7407F11003614819464F
:1006A000FFF724FE4FF416533B604FF00003BB806E
:1006B0004FF00003FB804FF000033B814FF000033D
:1006C000BB814FF00C037B813B465748194600F035
:1006D00095F955484FF0010100F068FA02E000BFBB
:1006E00000E000BF504B1B889BB203F02003002B9F
:1006F000F5D04D4B9B889BB27B757B7DA3F130037E
:100700000F2BEED801A252F823F000BF4D070008CE
:100710005B070008690700087707000885070008DD
:1007200093070008A1070008AF070008BD070008ED
:10073000CB070008E3060008E3060008E30600080C
:10074000E3060008E3060008D9070008344B344AE2
:10075000D26882F00102DA605FE0314B304AD26841
:1007600082F00202DA6058E02D4B2D4AD26882F006
:100770000402DA6051E02A4B294AD26882F008026A
:10078000DA604AE0264B264AD26882F01002DA602C
:1007900043E0234B224AD26882F02002DA603CE038
:1007A0001F4B1F4AD26882F04002DA6035E01C4BD2
:1007B0001B4AD26882F08002DA602EE0184B184A99
:1007C000D26882F48072DA6027E0154B144AD2684E
:1007D00082F40072DA6020E01448FFF701FF4FF066
:1007E0000103FB8211E00E4BDA68FB8A02EA030385
:1007F000002B03D00E48FFF7F3FE02E00D48FFF791
:10080000EFFEFB8A4FEA4303FB82FB8AB3F5007FCE
:10081000E9D90948FFF7E4FE00BF63E700023000B2
:10082000000C01400008014000380140EC0B0008BA
:10083000000C0008040C0008080C000880B489B003
:1008400000AF78604FF00003FB614FF00003BB6125
:100850004FF000037B614FF000033B614FF000035A
:10086000FB60504B5B6803F00C03FB61FB69042BDE
:1008700007D0082B09D0002B32D17B684A4A1A6076
:1008800032E07B68484A1A602EE0464B5B6803F40E
:100890007013BB61434B5B6803F480337B61BB69BE
:1008A0004FEA934303F10203BB617B69002B06D13E
:1008B000BB693E4A02FB03F27B681A6014E0394BC5
:1008C000DB6A03F00F0303F10103FB60364AFB68A8
:1008D000B2FBF3F3BA6902FB03F27B681A6003E030
:1008E0007B68314A1A6000BF2E4B5B6803F0F0034F
:1008F000FB61FB694FEA1313FB612D4AFB69D318B7
:100900001B78DBB23B617B681A683B6922FA03F211
:100910007B685A60234B5B6803F4E063FB61FB690F
:100920004FEA1323FB61224AFB69D3181B78DBB221
:100930003B617B685A683B6922FA03F27B689A60E4
:10094000184B5B6803F46053FB61FB694FEAD323E8
:10095000FB61174AFB69D3181B78DBB23B617B68EC
:100960005A683B6922FA03F27B68DA600D4B5B68D8
:1009700003F44043FB61FB694FEA9333FB610D4A8B
:10098000FB69D3181B78DBB23B617B68DA683B6993
:10099000B2FBF3F27B681A6107F12407BD4680BC05
:1009A000704700BF0010024000127A0000093D00AD
:1009B000000000201000002080B483B000AF7860F9
:1009C0000B46FB70FB78002B07D00B4B0A4A916952
:1009D0007A6841EA02029A6108E0074B064A916987
:1009E0007A686FEA020201EA02029A6107F10C07D3
:1009F000BD4680BC704700BF0010024080B58CB07F
:100A000000AF786039604FF00003FB624FF00003E5
:100A1000BB624FF000037B624FF000033B624FF07C
:100A20000003FB617B68FB617B681B8A9BB2FB62F6
:100A3000FA6A4CF6FF7302EA0303FB623B68DB8849
:100A4000FA6A42EA0303FB62FB6A9AB27B681A8283
:100A50007B689B899BB2FB62FA6A4EF6F31302EA4B
:100A60000303FB623B689A883B681B8942EA0303E5
:100A70009AB23B685B8942EA03039BB2FA6A42EA94
:100A80000303FB62FB6A9AB27B689A817B689B8A4C
:100A90009BB2FB62FA6A4FF6FF4302EA0303FB6272
:100AA0003B689B89FA6A42EA0303FB62FB6A9AB2DB
:100AB0007B689A8207F108031846FFF7BFFEFA69C0
:100AC000384B9A4202D17B69BB6201E03B69BB6251
:100AD0007B689B899BB29BB21BB2002B0FDABA6A70
:100AE00013464FEA83039B184FEA83029A183B6828
:100AF0001B684FEA4303B2FBF3F37B620EE0BA6A72
:100B000013464FEA83039B184FEA83029A183B6807
:100B10001B684FEA8303B2FBF3F37B627A6A224BD2
:100B2000A3FB02134FEA53134FEA0313FB62FB6A62
:100B30004FEA13134FF0640202FB03F37A6AD31AED
:100B40003B627B689B899BB29BB21BB2002B10DA85
:100B50003B6A4FEAC30303F13202134BA3FB0213B8
:100B60004FEA531303F00703FA6A42EA0303FB62F6
:100B70000FE03B6A4FEA031303F132020A4BA3FB77
:100B800002134FEA531303F00F03FA6A42EA030316
:100B9000FB62FB6A9AB27B681A8107F13007BD4697
:100BA00080BD00BF003801401F85EB5180B483B089
:100BB00000AF78600B46FB70FB78002B08D07B6899
:100BC0009B899BB243F400539AB27B689A8107E0F9
:100BD0007B689B899BB223F400539AB27B689A810D
:100BE00007F10C07BD4680BC704700BF3D3D3D4C42
:100BF0004544732073746174653A3D3D3D000000C7
:100C00004F4E00004F4646003D3D3D3D3D3D3D3D84
:0C0C10003D3D3D3D3D3D3D3D3D000000B3
:100C1C000000000001020304010203040607080996
:040C2C0002040608B0
:0400000508000000EF
:00000001FF
